:0200000480007A
:10000000971000009380000013012000930130003E
:10001000130240009302500013036000930370002A
:1000200013048000930490001305A0009305B00012
:100030001306C0009306D0001307E0009307F000FA
:1000400013080001930810011309200193093001DE
:10005000130A4001930A5001130B6001930B7001C6
:10006000130C8001930C9001130DA001930DB001AE
:10007000130EC001930ED001130FE001930FF00196
:100080001300000013000000130000001300000024
:10009000130000001300000023A0000023A2200092
:1000A00023A4300023A6400023A8500023AA600008
:1000B00023AC700023AE800023A0900223A2A002F4
:1000C00023A4B00223A6C00223A8D00223AAE002E0
:1000D00023ACF00223AE000323A0100523A22005C9
:1000E00023A4300523A6400523A8500523AA6005B4
:1000F00023AC700523AE800523A0900723A2A007A0
:1001000023A4B00723A6C00723A8D00723AAE0078B
:1001100023ACF00797110000938181F617040000CB
:100120001300000013000000130000001300000083
:100130001300000097040000B384844023A09100C2
:1001400017150000130505EC97150000938585F33E
:10015000370610F01306C6F26306B5028326C50003
:100160002320D600832685002320D6008326450041
:100170002320D600832605002320D6001305050181
:100180006FF09FFD370510F0130505F223200500E1
:04019000000000006B
:10100000FFFFFFFFFFFFFFFFFFFFFFFFFFFFFFFFF0
:10101000FFFFFFFFFFFFFFFFFFFFFFFFFFFFFFFFE0
:10102000FFFFFFFFFFFFFFFFFFFFFFFFFFFFFFFFD0
:10103000FFFFFFFFFFFFFFFFFFFFFFFFFFFFFFFFC0
:10104000FFFFFFFFFFFFFFFFFFFFFFFFFFFFFFFFB0
:10105000FFFFFFFFFFFFFFFFFFFFFFFFFFFFFFFFA0
:10106000FFFFFFFFFFFFFFFFFFFFFFFFFFFFFFFF90
:10107000FFFFFFFFFFFFFFFFFFFFFFFFFFFFFFFF80
:040000058000000077
:00000001FF
